:020000040800F2
:1000000008060020190B00086D0400086D040008A4
:100010006D0400086D0400086D0400086D040008FC
:100020006D0400086D0400086D0400086D040008EC
:100030006D0400086D0400086D0400086D040008DC
:100040005101000851010008510100085101000848
:100050005101000851010008510100085101000838
:10006000510100085101000851010008F90400087D
:100070005101000851010008510100085101000818
:100080005101000851010008510100085101000808
:1000900051010008510100085101000851010008F8
:1000A00051010008510100085101000851010008E8
:1000B000510100085101000899040008510100088D
:1000C00051010008510100085101000851010008C8
:1000D00051010008510100085101000851010008B8
:1000E00051010008510100085101000851010008A8
:1000F0005101000851010008510100085101000898
:100100005101000851010008510100085101000887
:100110005101000851010008510100085101000877
:100120005101000851010008510100085101000867
:100130005101000851010008510100085101000857
:100140005101000851010008510100085101000847
:100150002DE9F04F684600F063B80000EFF3088126
:1001600081F30988022181F31488BFF36F8F104B4C
:1001700083F308880F4B104A9A605A6942F404725C
:100180005A615A6A42F4E0225A624FF07F42DA61C1
:100190004FF47F021A62BFF34F8FBFF36F8F6FF080
:1001A0007F42A3F54F635A6001221A60704700BF77
:1001B0000802002000ED00E000000008054A9368F6
:1001C00091685B1A23F07F43984202D9C01A0B460C
:1001D000F6E7704710E000E04FF47A7300EBC000E0
:1001E000B0FBF3F0FFF7EABF00EBC000FFF7E6BF9C
:1001F00042F228335843FFF7E1BF08B572B605480D
:1002000000F058FABFF34F8FBFF36F8F024B034AD2
:10021000DA60FEE7F80D000800ED00E00400FA05E2
:10022000F7B50446EFF30382006AD2B2410704F146
:10023000240341D5EFF309851E4605F120070F2A57
:1002400040D82249DFF8A8C010F0080F204808BFA6
:100250006046AB6900901F4800F02CFAEB681E481E
:100260000093D5E90123296800F024FAE3682168A6
:1002700000931A48D4E9012300F01CFAE3692169CC
:1002800000931748D4E9052300F014FA236A29697A
:1002900013F0040FAB6918BF3A46009308BF32460B
:1002A0006B69104800F006FA3A463146EB690E4891
:1002B00000F000FAFFF7A1FFEFF309871D4604F1F4
:1002C0004406BCE70949103ABCE700BF0A0E000823
:1002D000140E0008230E0008470E0008770E0008D1
:1002E000A70E0008D70E0008070F0008060E00082A
:1002F0001B0E0008044B186880EA403080EA50402A
:1003000080EA40101860704700000020012208B504
:10031000064B07481A7000F0CDF94FF48052054B98
:100320001A614FF40052C3F8102408BD08060020DB
:100330002B0F0008000C014010B1024800F0BAB9C0
:10034000E4E700BF370F000810B50446114800F07D
:10035000B1F9002323601023A36040F2247363608B
:1003600040F201432360A368102B05D12368012BC1
:1003700002D1094800F09EF9A368102B08D140F281
:1003800001432068C31A58425841BDE81040D3E7E2
:100390000020FAE73B0F00084D0F000810B5044697
:1003A0000A4800F087F941F61F430122A36241F297
:1003B0008733E362E2600022626005222260E06A25
:1003C000BDE81040C31A58425841B5E75B0F00081A
:1003D0002DE9F0410D46074611461F4800F06AF925
:1003E0004FF0000801234FF480621C4E122173600D
:1003F0002846C6F8088077613561F26000F0A9F8F8
:1004000044F2D303164CC4F80480B3606368002B35
:10041000FCD06368012B04DD61681248013900F0EB
:1004200049F94FF480622946384600F0DFF810B1F0
:100430000D4800F03FF96368012B0BD14FF4806247
:100440002946384600F0D2F8B0FA80F04009BDE8FD
:10045000F04171E70020FAE76D0F0008000002404C
:10046000080600207E0F00089A0F000808B5EFF379
:10047000038172B60648C9B200F01CF94FF48052ED
:10048000044B1A614FF40052C3F81024FEE700BF7A
:10049000A60F0008000C01400022124B1A61124AFC
:1004A00013784BB14FF08042104BC3F88020BFF35C
:1004B0004F8FBFF36F8F7047137A0D49002B14BF16
:1004C0004FF480504FF08050086114BF4FF400503B
:1004D0004FF0005083F00103C1F810040548137277
:1004E00000F0E8B8000800400806002000E100E045
:1004F000000C0140221100080122044B5A60002226
:100500009A60034A53680133536070470000024009
:10051000080600202DE9F007B1E8F807A0E8F80781
:10052000203AF9D1BDE8F00770472DE9F007CDB2C8
:100530004FF001346C432346254626462746A04605
:10054000A146A246A0E8F807203AFBD1BDE8F00793
:100550007047F8B532F01F0506460F4614460CD01A
:1005600083070AD12A46FFF7E0FF04F01F0472193F
:100570001444A24203D13046F8BD3246F8E702F8EF
:10058000017BF6E7F8B532F01F0706460D46144624
:1005900010D040EA01039B070CD13A46FFF7BAFF9F
:1005A0003D44F31904F01F04013B2C44A54203D140
:1005B0003046F8BD3346F7E715F8012B03F8012F55
:1005C000F4E7884230B405460C4602D230BCFFF74F
:1005D000D9BF034614448218934202D1284630BC46
:1005E000704714F8011D02F8011DF5E7034610B528
:1005F00002449A4201D1002005E013F8010B11F8E2
:10060000014B001BF5D010BD03460246D01A12F86C
:10061000011B0029FAD1704703460020884201D00F
:100620001A5C02B970470130F8E770B5054600243E
:10063000A24201D1002006E02E5D0B5DF01A02D12E
:100640000134002EF4D170BD6FF00042FFF7EDBF12
:10065000421E11F8013B02F8013F002BF9D170470F
:1006600070B502460B46EFF3108404F0010472B635
:100670000D2580210D4800F063F80C490C4A11F853
:10068000013B13B904B962B670BD0A2B07D00D2B1C
:10069000F5D01668360607D55360F0E700BF166838
:1006A0003606FBD55560F4E700BFF2E711060020DF
:1006B000003801400FB407B504A951F8040B0191AB
:1006C000FFF7CEFF03B05DF804EB04B0704710B540
:1006D0000B4A0C4C9369204643F4804393610922F2
:1006E000114600F0A3F918220A21204600F09EF9D5
:1006F00040F27122044B9A6042F20C02DA6010BDA3
:10070000001002400008014000380140064B5A68C2
:10071000DA6842F02002DA600022044B83F82523D5
:1007200020225A60704700BF0038014000E100E01D
:1007300003688B4238BF1A70036801330360704747
:100740002DE9F04F8046174687B01D464B1E02909C
:100750000093C118BA461AF8012B52B9029B8B427A
:1007600000F2FA801A700298A0EB080007B0BDE80A
:10077000F08F252A04D002A8FFF7DAFF5746E9E7F1
:10078000002634461CE0A2F16303152B26D8DFE8CF
:1007900003F072562525253E562525252525491188
:1007A00025255B2558252511392A21D9582A15D107
:1007B00044F4807444F0100436E055F8046BBA46F3
:1007C000574617F8012B782A08D8622ADBD8302A36
:1007D0000BD0E9D8232A05D02A2AEED002A8FFF7A9
:1007E000A7FFB7E744F48064E9E744F40064E6E770
:1007F000A2F130063A4612F8013BA3F13000092875
:10080000DDD80A2000FB06361746303EF2E79AF89C
:100810000130682B06BF44F480540AF1020744F407
:100820000054CCE744F00804E30455F8049B04F4B6
:10083000007224D55FFA89F924F4007432E044F49C
:10084000007444F00A04EFE755F8044B2644A6EB85
:10085000040A14F8012B52B9BAF1000F7FF77AAFEE
:10086000202202A8FFF764FF0AF1FF3AF4E702A88A
:10087000FFF75EFFEBE755F8042BD2B2AEE7A0041A
:1008800037D59AB30FFA89F9B9F1000FD4DA2305F5
:1008900005D52D2202A8FFF74BFF24F40074013E7A
:1008A000C9F1000960050FD504F01F0ABAF1080F5D
:1008B00002D0BAF1100F07D1302202A8FFF738FF9B
:1008C000BAF1100F18D0013E0DF10C0AB9F1000F6A
:1008D00018D130230DF10D0B8DF80C3014F4006F8E
:1008E00014BF30222022ABEB0A0327E01FFA89F95C
:1008F000A2E7002AA0D0C7E7782202A8FFF718FFD6
:10090000023EE1E7D346174A14F4807F164808BF39
:10091000104604F01F02B9FBF2FC02FB1C9E10F80B
:100920000EE00BF801EBCE467245E146F3D9D5E770
:1009300002A80193FFF7FCFE019B013EB342F7DBE7
:10094000A30503D52D2202A8FFF7F2FED3453FF4FD
:1009500001AF1BF8012DF6E788459CBF009B08F806
:10096000032000E735110008241100080CB407B576
:1009700004AB53F8042B0193FFF7E2FE03B05DF8DC
:1009800004EB02B0704700BF08B5FFF7E7FB122287
:10099000234B1A60A3F580531A6842F480321A6020
:1009A0001A68910335D51F4A5A601A6842F080725E
:1009B0001A601A6892012ED55A6842F002025A60F3
:1009C0005A6802F00C02082A27D11A6822F00102A4
:1009D0001A600722DA6140F61D029A6101225A610B
:1009E0004FF08062104B5A604FF0443302F1705266
:1009F00002F5843253601360C2F80434C2F8003444
:100A0000C2F80438C2F80038BFF34F8FBFF36F8FBE
:100A100008BD00BFC4E700BFCBE700BFD0E700BF01
:100A20000020024000C41D0000000140130914BF53
:100A300001234FF48033072903FA01F330B5036132
:100A40004FF00F0402F00F020AD9083945688B00F5
:100A50009C4025EA040402FA03F32343436030BDBB
:100A6000036889008C4023EA040402FA01F121435F
:100A70000160F4E7044AD36813F00103FBD1342189
:100A8000D1601361704700BF00200240094B1A6813
:100A900042F001021A601A68910709D5064B1A69DB
:100AA000120641BF054A5A6002F188325A60E1E7F6
:100AB00000BFF0E70010024000200240230167451C
:100AC00008B5FFF7D7FF064B1A6942F002021A6118
:100AD00058611A6942F040021A61BDE80840C9E74E
:100AE0000020024070B50C461546FFF7C3FF094EC3
:100AF0002D1A0444844205EB000200D170BD336915
:100B000043F00103336130F8023B1380FFF7B2FF7B
:100B1000F0E700BF00200240F0B58D488D4985B058
:100B2000884203D08C4A121AFFF72CFD8B488C4D5B
:100B30008C4C00212A1AFFF70CFDFFF725FFE36913
:100B4000894E43F0C053E361FFF7C1FD8748FFF7CB
:100B5000B1FD8748FFF7AEFD8648FFF7ABFD1622D3
:100B60000C218548FFF762FF16220D218348FFF70D
:100B70005DFF834B8348844F19885A8804331B8850
:100B8000008836883F8880B2B6B2BFB292B2CDE953
:100B9000016700909BB289B27C48FFF78BFD7C4BCC
:100BA0007C48198889B2FFF785FD7B4B7B481E681E
:100BB000C6F30B01FFF77EFD7948310CFFF77AFD94
:100BC00016B17848FFF776FD032640F64D37E36906
:100BD000012143F40013E3617348FFF7B5FBE369B8
:100BE000022143F48003E3617048FFF7ADFBA36982
:100BF000012143F48053A3616D48FFF75BFD6D4B0A
:100C00005E601F605868831B58425841FFF794FB91
:100C1000E369022143F48043E3616548FFF74AFD3D
:100C2000654B40245E601F605868821B50425041F3
:100C3000FFF782FB01216148FFF7B0FB02214FF073
:100C40008040FFF7ABFB31465D48FFF7A7FB04216F
:100C50005C48FFF7A3FB01224FF400615A4B5A6036
:100C60005A4B83F80B43C3F88011594819603C492B
:100C7000FFF7AEFB02223A495648FFF7A9FB32467E
:100C800055495348FFF7A4FB544E0422524951489A
:100C9000FFF79EFB21465248FFF70CFDFFF7F6FEDB
:100CA0003046FFF70DFF4FF48062FF212C48FFF71D
:100CB00050FC4FF4806230462949FFF797FC044608
:100CC00000283CD1FFF716FB28510434B4F5806F9F
:100CD000F8D1324621462248FFF704FF2246204938
:100CE0003E48FFF783FC50BB3E48FFF7E3FC3E481D
:100CF000FFF7E0FC4022354B83F81E234FF0804283
:100D0000C3F8802137481A60FFF7D4FC1421374814
:100D1000FFF7D0FC124D3649364C2A460E68A242E7
:100D200010D32A460E60A242F7D252F8046BFFF7A6
:100D3000E1FA8642F7D0FFF7E9FA72B6FEE7FFF76D
:100D4000E5FAD4E7FFF7D6FA42F8040BE7E700BF6D
:100D500000000020481100080400002008060020C0
:100D60009406002000100240F0F7FF1FC20F000899
:100D7000D60F0008FB0F0008000C014000100140D6
:100D8000E8F7FF1FEEF7FF1FF2F7FF1F251000081F
:100D9000E0F7FF1F4D100008002004E0611000087C
:100DA00075100008891000080054004000580040E9
:100DB000C31000080030014000380040002C014002
:100DC00000040040000800400000024000E100E094
:100DD00000000008010000089506002000FC000843
:100DE000D5100008370F0008EC10000800110008AB
:100DF0000000002000500020526573657474696E15
:100E0000672E2E2E0A004952510045786365707492
:100E1000696F6E005468726561640048616E646C4D
:100E2000657200556E65787065637465642025731E
:100E3000202325752061742050433D2530387820CB
:100E4000282573293A0A002072303A2020253038AC
:100E50007820202072313A20202530387820202038
:100E600072323A20202530387820202072333A2000
:100E700020253038780A002072343A202025303876
:100E80007820202072353A20202530387820202004
:100E900072363A20202530387820202072373A20C8
:100EA00020253038780A002072383A202025303842
:100EB0007820202072393A202025303878202020D0
:100EC0007231303A20253038782020207231313A82
:100ED00020253038780A00207231323A2025303807
:100EE0007820202073703A20202530387820202068
:100EF0006C723A20202530387820202070633A2008
:100F000020253038780A00206D73703A202530385B
:100F1000782020207073703A2025303878202020E7
:100F20007073723A20253038780A002A2A464149DF
:100F30004C45442A2A0A004F4B0A005465737469D1
:100F40006E672049324325642E2E2E20005B4661B9
:100F50006B6520436869703F5D2000546573746958
:100F60006E672054494D25642E2E2E2000444D419D
:100F70002054657374202325752E2E2E20005B537C
:100F8000707572696F7573204952513A2046616BD2
:100F90006520436869703F5D20005B4261642044C6
:100FA0006174615D20002A2A4641494C45442A2A41
:100FB000205B457863657074696F6E202325755DCD
:100FC0000A000A2A2A20426C696E6B7920546573E4
:100FD00074202A2A0A002A2A204B65697220467248
:100FE00061736572203C6B6569722E78656E40672F
:100FF0006D61696C2E636F6D3E0A002A2A20687449
:101000007470733A2F2F6769746875622E636F6D01
:101010002F6B656972662F477265617365776561CD
:101020007A6C650A0053657269616C203D20253039
:1010300034783A253034783A253034783A253034CB
:10104000783A253034783A253034780A00466C6195
:1010500073682053697A6520203D2025756B420A0C
:1010600000446576696365204944203D2030782539
:101070003034780A005265766973696F6E20203DBE
:10108000203078253034780A002A2A5741524E49B8
:101090004E472A2A3A2031307878382F422064652A
:1010A000766963652072657475726E656420766119
:1010B0006C6964204944434F4445212046616B6577
:1010C0003F0A0054657374696E6720535049256464
:1010D0002E2E2E200054657374696E672025756B63
:1010E0004220466C6173682E2E2E2000456E616290
:1010F0006C652054494D34204952512E2E2E20002B
:1011000054657374696E672025756B422053524194
:101110004D2028656E646C657373206C6F6F702949
:101120002E2E2E00303132333435363738394142A5
:10113000434445460030313233343536373839612F
:081140006263646566000000B3
:041148003C26A28718
:0400000508000000EF
:00000001FF
